:020000040000FA
:100000000C9463000C948B000C948B000C948B006C
:100010000C948B000C948B000C948B000C948B0034
:100020000C948B000C948B000C948B000C948B0024
:100030000C948B000C948B000C948B000C948B0014
:100040000C94090B0C948B000C94790B0C94530BAF
:100050000C948B000C948B000C948B000C948B00F4
:100060000C94AB0B0C948B000000000023002600C6
:10007000290000000008000201000003040700003E
:1000800000000000000000000000250028002B00F8
:1000900000000000240027002A00040404040404D3
:1000A0000404020202020202030303030303010227
:1000B00004081020408001020408102001020408F6
:1000C0001020CA0C411111241FBECFEFD8E0DEBFB3
:1000D000CDBF11E0A0E0B1E0EAEBF9E202C005908B
:1000E0000D92AE3AB107D9F723E0AEEAB1E001C014
:1000F0001D92AB35B207E1F710E0C2E6D0E004C0D4
:100100002197FE010E94A513C136D107C9F70E94AD
:100110001F0D0C94D0140C94000008950895CF93F3
:10012000DF9390E0FC01E255FF4F249186569F4FEC
:10013000FC0184918823C1F090E0880F991FFC0195
:10014000E057FF4FC591D491FC01EA57FF4FA591AD
:10015000B4919FB7F8943881822F80958323888348
:10016000EC91E22BEC939FBFDF91CF910895833008
:1001700081F028F4813099F08230A9F00895873019
:10018000A9F08830C9F08430B1F4809180008F7D6F
:1001900003C0809180008F7780938000089584B59C
:1001A0008F7784BD089584B58F7DFBCF8091B0009B
:1001B0008F778093B00008958091B0008F7DF9CF44
:1001C000CF93DF93282F30E0F901EE58FF4F849151
:1001D000F901E255FF4FD491F901E656FF4FC49162
:1001E000CC23A1F081110E94B700EC2FF0E0EE0FBC
:1001F000FF1FE859FF4FA591B491EC91ED2381E0E9
:1002000090E009F480E0DF91CF91089580E090E0E4
:10021000FACF1F93CF93DF93282F30E0F901EE58E8
:10022000FF4F8491F901E255FF4FD491F901E65651
:10023000FF4FC491CC23A9F0162F81110E94B70063
:10024000EC2FF0E0EE0FFF1FEA57FF4FA591B4919E
:100250008FB7F894EC91111108C0D095DE23DC9390
:100260008FBFDF91CF911F910895DE2BF8CF8230A1
:10027000910538F0880F991F880F991F05970197EE
:10028000F1F708953FB7F8948091370290913802C2
:10029000A0913902B0913A0226B5A89B05C02F3F24
:1002A00019F00196A11DB11D3FBFBA2FA92F982F9C
:1002B0008827BC01CD01620F711D811D911D42E097
:1002C000660F771F881F991F4A95D1F708958F925F
:1002D0009F92AF92BF92CF92DF92EF92FF924B012B
:1002E0005C010E9442016B017C010E9442016C1979
:1002F0007D098E099F09683E734081059105A8F329
:1003000021E0821A9108A108B10888EEC80E83E0A6
:10031000D81EE11CF11C81149104A104B10429F739
:10032000FF90EF90DF90CF90BF90AF909F908F9015
:100330000895AF92BF92CF92DF92EF92FF920F9308
:100340001F93CF93DF936C017B018B01040F151F6B
:10035000EB015E01AE18BF08C017D10759F06991D3
:10036000D601ED91FC910190F081E02DC601099537
:10037000892B79F7C501DF91CF911F910F91FF90E4
:10038000EF90DF90CF90BF90AF900895FC01538D18
:10039000448D252F30E0842F90E0821B930B54175F
:1003A00010F0CF96089501970895FC01918D828DEC
:1003B000981761F0A28DAE0FBF2FB11D5D968C9185
:1003C000928D9F5F9F73928F90E008958FEF9FEFC4
:1003D0000895FC01918D828D981731F0828DE80F80
:1003E000F11D858D90E008958FEF9FEF0895FC013A
:1003F000918D228D892F90E0805C9F4F821B910907
:100400008F739927089581E992E00E94F70121E016
:10041000892B09F420E0822F089580E090E0892B59
:1004200029F00E94030281110C9400000895FC0140
:10043000A48DA80FB92FB11DA35ABF4F2C91848D45
:1004400090E001968F739927848FA689B7892C93A2
:10045000A089B1898C91837080648C93938D848DF5
:10046000981306C00288F389E02D80818F7D8083F8
:100470000895EF92FF920F931F93CF93DF93EC01B8
:1004800081E0888F9B8D8C8D98131AC0E889F9893B
:10049000808185FF15C09FB7F894EE89FF8960833E
:1004A000E889F98980818370806480839FBF81E0BF
:1004B00090E0DF91CF911F910F91FF90EF90089501
:1004C000F62E0B8D10E00F5F1F4F0F731127E02EDC
:1004D0008C8D8E110CC00FB607FCFACFE889F98914
:1004E000808185FFF5CFCE010E941702F1CFEB8D01
:1004F000EC0FFD2FF11DE35AFF4FF0829FB7F894E8
:100500000B8FEA89FB8980818062CFCFCF93DF9305
:10051000EC01888D8823B9F0AA89BB89E889F9891B
:100520008C9185FD03C0808186FD0DC00FB607FC50
:10053000F7CF8C9185FFF2CF808185FFEDCFCE0183
:100540000E941702E9CFDF91CF910895FC018385C6
:100550008F3F19F061E00C9409010895FC0180813E
:100560009181892B39F0A281B3819C9111968C9154
:100570009CBD8DBD83858F3F19F060E00C9409010F
:100580000895AF92BF92CF92DF92EF92FF920F93B6
:100590001F93CF93DF93EC0188819981892B89F098
:1005A0006EBD0DB407FEFDCFBEB48B2DDF91CF9194
:1005B0001F910F91FF90EF90DF90CF90BF90AF9081
:1005C00008958885998511E0892B09F010E8AA24FF
:1005D000A394862F812309F0A12C062F2C813D8125
:1005E0004E815F8160E271EA87E090E00E948313B0
:1005F000F22EB02EE12CC22ED12CFF2019F0C60114
:100600000E9437018A85877F09F042C08D858F3F20
:1006100089F0902F912381E009F480E08A1551F050
:10062000EF85F8898F89992369F19081892B8083DF
:10063000AA24A394E989FA898081998D892B8083E2
:10064000FF2019F0C6010E9437018E858F3F39F0D7
:10065000EB89FC898081988D892309F0E12AE98959
:10066000FA899081898D8095892380838E858F3F3B
:1006700009F0BE2C88859985892BB9F5110F1111C8
:10068000BCCF93CF9081809589238083A12CD2CF3A
:10069000E989FA898081998D892B8083FF2019F05F
:1006A000C6010E9437018D858F3F49F0EF85F8899B
:1006B0008F89902F9123A9F09081892B8083E989DC
:1006C000FA899081898D8095892380838E858F3FDB
:1006D00069F2EB89FC898081988D892339F2E12ABE
:1006E000C5CF908180958923E9CF1695C8CF8F9289
:1006F0009F92AF92BF92CF92DF92EF92FF920F93B1
:100700001F93CF93DF937C014B016A01B22EA32E7E
:100710000E94AE02E401C80CD91CCC15DD0569F4B9
:10072000CB2DDA2D0C0F1D1FC017D10759F06FEF1D
:10073000C7010E94C1028993F7CF6991C7010E9446
:10074000C102EBCFC7010E94A60281E0DF91CF91E9
:100750001F910F91FF90EF90DF90CF90BF90AF90DF
:100760009F908F9008958F929F92AF92BF92CF9259
:10077000DF92EF92FF920F931F93CF93DF937C0151
:10078000B62EA72E6A0149010E94AE02E401080DAF
:10079000191DC017D10761F4CB2DDA2DCC0EDD1E4B
:1007A000CC15DD0551F06991C7010E94C102F8CF57
:1007B0006991C7010E94C102ECCFC7010E94A60245
:1007C00081E0DF91CF911F910F91FF90EF90DF902B
:1007D000CF90BF90AF909F908F90089508952091F3
:1007E000CF01260F3327331F21323105ECF420913E
:1007F0006702FC0190E080E0243069F082E0089517
:10080000A091CF012191AC0141555E4FA40FB52FAE
:10081000B11D2C930196861798F38091CF01680F34
:100820006093CF0180E0089581E0089510926702FF
:1008300081E0809366021092410261E082E10E94B1
:10084000090161E083E10E940901E9EBF0E08081A8
:100850008E7F808380818D7F808388E48093B80041
:1008600085E48093BC0008951092400210923F02EC
:1008700010926E02109290020E9416048DE890E091
:1008800090933E0280933D028EE890E090933C026C
:1008900080933B020895CF93DF9391E09093AE0154
:1008A0008823B9F0C091B800D091BA008091BC0003
:1008B0008A7B8093BC0060E082E10E94090160E0D5
:1008C00083E10E9409010E941604D093BA00C093EC
:1008D000B800DF91CF9108958F929F92AF92BF920F
:1008E000CF92DF92EF92FF920F931F93CF93DF93FC
:1008F000D0919002D13208F0D7C0182FC0918F024A
:100900000E9442016B017C018091670281116BC0E2
:1009100082E080936702109366028FEF80936502F6
:1009200010926402D0936302AFE6B2E0E3E4F2E037
:1009300080E0D81391C01092420280914202CC0F05
:10094000C82BC093420280914102813009F088C0D7
:10095000109241020E9442016B017C01809142028F
:100960008093BB008091690290916A02A0916B0212
:10097000B0916C02892B8A2B8B2BA1F00E94420133
:100980000091690210916A0220916B0230916C0211
:100990006C197D098E099F09061717072807390763
:1009A00008F442C08091BC0083FDD8CF85EC8093D1
:1009B000BC000E9442016B017C0180916702823081
:1009C00009F450C0809165028F3F09F46FC0809197
:1009D0006502803209F46CC080916502803309F4AD
:1009E00069C084E026C08091690290916A02A0915A
:1009F0006B02B0916C02892B8A2B8B2B09F484CF6C
:100A00000E9442018090690290906A02A0906B025D
:100A1000B0906C026C197D098E099F0986169706A5
:100A2000A806B90608F070CF809168020E944B04B6
:100A300085E010926E021092900210926D02DF918A
:100A4000CF911F910F91FF90EF90DF90CF90BF90CB
:100A5000AF909F908F9008959D9191938F5F69CFF4
:100A600085EEA5CF8091690290916A02A0916B02F8
:100A7000B0916C02892B8A2B8B2B09F49ECF0E949C
:100A800042010091690210916A0220916B0230913B
:100A90006C026C197D098E099F0906171707280734
:100AA000390708F08ACFC0CF81E0C3CF80E0C1CF43
:100AB00082E0BFCF83E0BDCF1F93CF93DF93162F8C
:100AC000CAE4D3E0AB85BC859C8121E020936D0214
:100AD00090938F0210926E0210929002ED91FC9111
:100AE00011970190F081E02D682FCD0109958B853C
:100AF0009C85DC01ED91FC910190F081E02D612F4E
:100B0000099581E0DF91CF911F910C946C04809145
:100B10004E036FEF803359F486E00E945C056FEF5F
:100B200087E00E945C056FEF88E00C945C0584E030
:100B30000E945C056FEF83E00E945C056FEF82E02E
:100B4000F4CF0F931F93CF93DF938C01EB01DC0164
:100B50001B968D919C9121E020936D022EE32093B2
:100B60008F0210926E0210929002DC01ED91FC91C6
:100B70000190F081E02D68810995F80183859485C5
:100B8000DC01ED91FC910190F081E02D69810995E6
:100B900081E0DF91CF911F910F910C946C04CF9362
:100BA000DF9300D0CDB7DEB790E899838A83BE018A
:100BB0006F5F7F4F8AE493E00E94A1050F900F9032
:100BC000DF91CF910895CF93DF9300D0CDB7DEB7FB
:100BD000882381F080EC90E899838A83BE016F5F5F
:100BE0007F4F8AE493E00E94A1050F900F90DF9160
:100BF000CF91089580E8EFCFCF93DF9300D0CDB7AA
:100C0000DEB720E429836A83BE016F5F7F4F0E94B5
:100C1000A10581E090E00F900F90DF91CF910895B2
:100C20001F93CF93DF93EA01122FDC0111968D9170
:100C30009C91DC01ED91FC910280F381E02D0995FE
:100C4000C817D90729F4812F0E946C0491E0811103
:100C500090E0892FDF91CF911F910895CF92DF927D
:100C6000EF92FF920F931F93CF93DF9300D0CDB7F6
:100C7000DEB7DC0151964D935D936D937C93549751
:100C80001C968C911C978823C1F11E964C931E973D
:100C9000452F562F672F7727882399F11D964C9360
:100CA0001D977D018DE0E80EF11C18969C91189718
:100CB00019968C91199799838A83CD90DC9011971E
:100CC000C114D10409F448C01B960C9110E098019E
:100CD0002E5F3F4FD60114968D919C9182179307FA
:100CE000A0F480E00F900F90DF91CF911F910F91B2
:100CF000FF90EF90DF90CF9008951D964C931D9735
:100D0000C7CF1E964C931E97CCCFF601818192815E
:100D1000208131E030936D0220938F0210926E0299
:100D2000109290020115110541F421E042E050E0DB
:100D3000B701C6010E941006D5CFDC01ED91FC91F0
:100D40000280F381E02DA801BE016F5F7F4F0995FE
:100D50000817190731F6E9CF1296ED91FC91139718
:100D6000309751F116962D913C9117971B960C9147
:100D700010E02330310579F48E7F89839A830F5FE9
:100D80001F4F9E012F5F3F4F42E050E0B701CF0160
:100D90000E94B303A7CF2115310519F49F779983DA
:100DA000F0CF2230310511F49068F9CF21303105B0
:100DB00041F79F779064F3CF1496ED91FC911597CE
:100DC000309709F48ECF8085882309F48ACFC680B6
:100DD000D780C114D10409F484CF02E010E0970158
:100DE0001B964C91BE016F5F7F4F81859285F60106
:100DF000099578CFCF93DF93EC018B818823A1F005
:100E0000888191E090936D0280938F0210926E0220
:100E10001092900281E00E946C0491E0811190E0B8
:100E2000892FDF91CF9108950E94340481E08B8354
:100E3000CE010E94FA06982F8111E2CFF1CF0895DA
:100E4000E091400280913F02E81730F4F0E0EE506C
:100E5000FE4F808190E008958FEF9FEF089590916D
:100E6000400280913F022FEF3FEF981748F4E92F9F
:100E7000F0E0EE50FE4F208130E09F5F9093400203
:100E8000C901089580913F0290914002891B990BFE
:100E90000895CF92DF92EF92FF920F931F93CF931B
:100EA000DF937C01CB018A0120916D02222389F01E
:100EB000EB016B01C40ED51ECC15DD0569F06991FF
:100EC000D701ED91FC910190F081E02DC7010995CA
:100ED000F3CF642F0E94EF03C801DF91CF911F91E0
:100EE0000F91FF90EF90DF90CF900895CF93DF9315
:100EF0001F92CDB7DEB7698320916D022223F9F0EE
:100F000020919002203258F021E030E0FC01338340
:100F1000228390E080E00F90DF91CF91089580913F
:100F20006E02E82FF0E0E159FD4F998190838F5FC9
:100F300080936E028093900281E090E0ECCF61E0BC
:100F4000CE0101960E94EF03F7CF90E080E0089574
:100F50002F923F924F925F926F927F928F929F92C9
:100F6000AF92BF92CF92DF92EF92FF920F931F93B7
:100F7000CF93DF9300D000D000D0CDB7DEB77C0197
:100F80007E836D830D969C838B83D70118969C91ED
:100F9000189719968C91199799838A83CD90DC9034
:100FA0001197C114D10409F450C11B964C9150E023
:100FB000F6018481958184179507A8F0808191E0DE
:100FC00090936D0280938F0210926E0210929002A5
:100FD00020E0BE016F5F7F4FC6010E941006712C9A
:100FE000612C81111AC080E026960FB6F894DEBFFE
:100FF0000FBECDBFDF91CF911F910F91FF90EF906A
:10100000DF90CF90BF90AF909F908F907F906F9028
:101010005F904F903F902F900895D60114968D9138
:101020009C9102E010E0061917098017910708F457
:101030008C01F60150800E9442014B015C018091BD
:101040006702811176C0B02EF0E2F01710F440E292
:10105000B42E81E08093670221E082E090E0801B63
:10106000910B6816790608F420E0209366029FEF42
:1010700090936502109264028FEF8B0D8093630250
:10108000A1E0A093420280914202550C582A50924E
:10109000420280914102813009F093C010924102D6
:1010A0000E9442011B012C01809142028093BB00EF
:1010B0008091690290916A02A0916B02B0916C02DA
:1010C000892B8A2B8B2BA1F00E944201209169026F
:1010D00030916A0240916B0250916C02621973095F
:1010E00084099509261737074807590708F442C0AD
:1010F0008091BC0083FDD8CFB5ECB093BC000E94BA
:1011000042011B012C0180916702813009F45DC00E
:10111000809164028B1510F4B0906402A3E4B2E0F5
:10112000E2EFF1E080E08B1551F19D9191938F5F9B
:10113000FACF8091690290916A02A0916B02B091FE
:101140006C02892B8A2B8B2B09F479CF0E944201E8
:101150002091690230916A0240916B0250916C02B9
:10116000681979098A099B0926173707480759071B
:1011700008F065CF809168020E944B04B12C109258
:101180004002B0923F02B016110609F02CCF8B80BE
:101190009C80860C971C5401C501881999098017F9
:1011A0009107A8F5D60111968D919C91DC01ED91E6
:1011B000FC910284F385E02D0995F50181935F018F
:1011C000EBCFE5EEE093BC009ACF8091690290915D
:1011D0006A02A0916B02B0916C02892B8A2B8B2B37
:1011E00009F491CF0E9442012091690230916A0274
:1011F00040916B0250916C02621973098409950940
:10120000261737074807590708F07DCFB3CF600E80
:10121000711EF2E06F16710408F4FFCED7011C9620
:101220008C911C97811165C01E968C911E9790E041
:10123000982F8827ED81FE81918380831D962C91C4
:10124000822B9183808381E0CFCE1296ED91FC9129
:101250001397309761F116962D913C9117971B9635
:101260004C9150E02330310591F4816089839A8359
:101270004F5F5F4F02E010E02B813C81BE016F5F4A
:101280007F4FCF010E9477038111C8CFADCE2115CA
:10129000310519F490689983EDCF2230310511F4AE
:1012A0009F77F9CF2130310529F7906CF4CFF70102
:1012B000A481B581109709F496CE18968C91189751
:1012C000882309F490CE1496CD90DC901597C11424
:1012D000D10409F488CE02E010E02B813C814385E3
:1012E000BE016F5F7F4F19968D919C91F601099514
:1012F000CBCF1D968C911D9790E0982F8827ED817C
:10130000FE81918380831E962C919ACFFB010190E0
:101310000020E9F73197AF01461B570BDC01ED9137
:10132000FC910280F381E02D09948F929F92AF92FD
:10133000BF92EF92FF920F931F93CF93DF93CDB79E
:10134000DEB7A1970FB6F894DEBF0FBECDBF7C010C
:10135000FA01CB0119A2223008F42AE08E010F5DB8
:101360001F4F822E912CB12CA12CBF01A5019401FD
:101370000E948313F901CA016A300CF5605DD8013F
:101380006E938D01232B242B252B79F790E080E0A1
:10139000109721F0BD01C7010E948609A1960FB6E2
:1013A000F894DEBF0FBECDBFDF91CF911F910F919B
:1013B000FF90EF90BF90AF909F908F900895695CE1
:1013C000DECF2F923F924F925F926F927F928F92D9
:1013D0009F92AF92BF92CF92DF92EF92FF921F93B4
:1013E000CF93DF93EC016A017B01722EAB01960172
:1013F000CB01B6010E947E136CE371E0811126C01F
:1014000046015701E894B7F82FEF3FEF4FE75FE74A
:10141000C501B4010E947E1381110CC02FEF3FEF74
:101420004FE75FE7C501B4010E94B41160E471E0C9
:10143000181664F02FEF3FEF4FE75FE4C701B601E6
:101440000E940C131816B4F464E471E0CE01DF912D
:10145000CF911F91FF90EF90DF90CF90BF90AF9012
:101460009F908F907F906F905F904F903F902F90C4
:101470000C9486092FEF3FEF4FE75FECC701B601F1
:101480000E94B41187FDE0CF20E030E0A901C70140
:10149000B6010E94B411312C212C87FF0DC0E881C8
:1014A000F9810190F081E02D6DE2CE0109951C01DA
:1014B000F7FAF094F7F8F09410E060E070E080E064
:1014C0009FE3711641F020E030E040E251E40E94D9
:1014D000B9111F5FF6CFA70196010E9448112B0199
:1014E0003C010E942B124B015C012AE0BC01A401CB
:1014F000CE010E9495097C01E20CF31C1123E1F15D
:10150000C501B4010E945A129B01AC01C301B20192
:101510000E9447114B015C01E881F9810190F08143
:10152000E02D6EE2CE010995E80EF91E115020F172
:1015300020E030E040E251E4C501B4010E94111303
:101540002B013C010E942B124B01B12CA12C2AE053
:10155000B501A401CE010E949509E80EF91EC5014E
:10156000B4010E945A129B01AC01C301B2010E9456
:1015700047114B015C01DACFC701DF91CF911F9179
:10158000FF90EF90DF90CF90BF90AF909F908F90A3
:101590007F906F905F904F903F902F9008950C94A4
:1015A000860985ED8093BC008091690290916A0262
:1015B000A0916B02B0916C020796A11DB11D23E0B2
:1015C000B695A795979587952A95D1F72091BC0058
:1015D00024FD03C010926702089540916902509162
:1015E0006A0260916B0270916C02452B462B472B6F
:1015F00069F30097A105B10541F02AE22A95F1F7B8
:1016000000C00197A109B109E1CF809168020C9453
:101610004B041F920F920FB60F9211242F933F93FA
:101620008F939F93AF93BF93809133029091340235
:10163000A0913502B09136023091320223E0230F9F
:101640002D3758F50196A11DB11D209332028093CC
:10165000330290933402A0933502B0933602809106
:10166000370290913802A0913902B0913A02019666
:10167000A11DB11D8093370290933802A0933902C7
:10168000B0933A02BF91AF919F918F913F912F916B
:101690000F900FBE0F901F90189526E8230F02960B
:1016A000A11DB11DD2CF1F920F920FB60F92112420
:1016B0002F933F934F935F936F937F938F939F935A
:1016C000AF93BF93EF93FF9381E992E00E941702DB
:1016D000FF91EF91BF91AF919F918F917F916F910A
:1016E0005F914F913F912F910F900FBE0F901F90E0
:1016F00018951F920F920FB60F9211242F938F936C
:101700009F93EF93FF93E091A102F091A202808159
:10171000E091A702F091A80282FD1BC09081809108
:10172000AA028F5F8F732091AB02821741F0E09184
:10173000AA02F0E0EF56FD4F958F8093AA02FF9129
:10174000EF919F918F912F910F900FBE0F901F904F
:1017500018958081F4CF1F920F920FB60F9211242B
:101760002F933F934F935F936F937F938F939F93A9
:10177000AF93BF93EF93FF938091B900887F80363A
:1017800009F44AC0F0F5883209F4A7C018F5803191
:1017900009F49BC0B8F4882309F4F9C0883009F42F
:1017A00094C0FF91EF91BF91AF919F918F917F91E5
:1017B0006F915F914F913F912F910F900FBE0F90BE
:1017C0001F901895883109F488C0803251F78093B2
:1017D000650214C0803409F49DC040F48033B9F32D
:1017E0008833F9F68093650285ECB0C0803509F442
:1017F00085C0883509F496C0883499F60E94D10ACC
:10180000D0CF883909F48CC038F5883729F050F4E6
:10181000883611F0803729F683E0809367021092B2
:10182000F10157C0883809F47BC0803919F080383D
:1018300009F0B7CF8091F101803208F071C0E091DA
:10184000F10181E08E0F8093F1018091BB00F0E007
:10185000EF52FE4F80833DC0803B39F0E0F4803A88
:1018600009F479C0883A09F09CCF84E0809367023C
:101870001092D0011092CF01E0913D02F0913E0212
:1018800009958091CF0181110FC081E08093CF0134
:101890001092AF0109C0803C09F4A6CF883C09F43E
:1018A000A3CF883B09F07DCFE091D00181E08E0F7E
:1018B0008093D001F0E0E155FE4F80818093BB0022
:1018C0009091D0018091CF0129C0809142028093F4
:1018D000BB0085EC8093BC0064CF90916402809142
:1018E0006302981758F5E091640281E08E0F8093AF
:1018F0006402F0E0ED5BFD4F8081E9CFE09164028E
:1019000081E08E0F809364028091BB00F0E0ED5B7C
:10191000FD4F808390916402809163029817C8F212
:1019200085E8D8CFE091640281E08E0F8093640255
:101930008091BB00F0E0ED5BFD4F808380916602FB
:1019400081115CCF81E08093410284EA8093BC00E6
:101950001092670226CF85EC8093BC00109267023C
:101960008091F101803230F4E091F101F0E0EF522A
:10197000FE4F10826091F10170E0E0913B02F09126
:101980003C0281ED91E009951092F1010ACF10928D
:10199000650234CFE1E9F2E01382128288EE93E02F
:1019A000A0E0B0E084839583A683B78320E131E093
:1019B0003183208325EC30E03587248724EC30E028
:1019C0003787268720EC30E0318B208B21EC30E00C
:1019D000338B228B22EC30E0358B248B26EC30E0ED
:1019E000378B268B118E128E138E148EEEE2F3E05F
:1019F0001382128284839583A683B78382E291E067
:101A000091838083EAE4F3E01382128284E391E01D
:101A10009183808315821682178210861186128622
:101A2000EAE3F3E01182108280E48383108611865A
:101A30001286138614861586168617860895CF9308
:101A4000DF93CDB7DEB7AC970FB6F894DEBF0FBE0D
:101A5000CDBF789484B5826084BD84B5816084BD37
:101A600085B5826085BD85B5816085BD80916E003C
:101A7000816080936E00109281008091810082606D
:101A800080938100809181008160809381008091AA
:101A900080008160809380008091B1008460809399
:101AA000B1008091B00081608093B00080917A0095
:101AB000846080937A0080917A00826080937A00BB
:101AC00080917A00816080937A0080917A008068AA
:101AD00080937A001092C10082E00E948F0083E020
:101AE0000E948F00E091A102F091A20282E0808327
:101AF000E0919D02F0919E021082E0919F02F09190
:101B0000A00280E180831092A902E091A502F091E9
:101B1000A60286E08083E091A302F091A402808176
:101B200080618083E091A302F091A40280818860AB
:101B30008083E091A302F091A40280818068808379
:101B4000E091A302F091A40280818F7D8083809137
:101B50003A0390913B03892BA9F486E090E00E9420
:101B6000AB13FC0180913D0380838EE293E092836E
:101B70008183138280E290E095838483F0933B031A
:101B8000E0933A03E0903A03F0903B030E94340460
:101B900011E0F7011383C7010E94FA06882309F4B4
:101BA0005BC080E090E1A0E0B0E080933E039093C2
:101BB0003F03A0934003B09341038AE090E0A0E08C
:101BC000B0E08093420390934303A0934403B09307
:101BD000450380E090E0A0E0B0E48093460390935A
:101BE0004703A0934803B093490380913A0390912F
:101BF0003B031FA218A619A61AA69F8B8E8B198EBF
:101C0000188E19A385E090E09F8F8E8F1AA302E0B3
:101C100008A340E050E160E070E0CE0146960E94EB
:101C20002E0680913A0390913B031A8A1B8A1C8AE4
:101C30001D8A9A8389831C821B821C871A861986B7
:101C40001D870B874FE959E360E070E0CE010196F4
:101C50000E942E0680933C038EE293E090935603FD
:101C6000809355030E94340480914F03982F98600D
:101C700090934F0312E01093530310925403EBE33D
:101C8000FDE03197F1F788620E94CF058BE496E47E
:101C90000197F1F780914F0380620E94CF0583E5A1
:101CA00092E00197F1F780914F0380620E94CF0587
:101CB00080914F0380620E94CF0584E0809350039F
:101CC0008CE00E94CF0581E00E94CF058BE39FE16D
:101CD0000197F1F71093510386E00E94CF0581E050
:101CE00080936D0210E310938F0210926E02109297
:101CF00090020E946C0481112DC210934E0367E084
:101D00000E945C058BE193E00197F1F765E184E0C7
:101D10000E945C050E9487050E94870564EF71E0C0
:101D200080E090E00E94670111E022E0822E912C79
:101D300002E035E0232E312C40E0A42E40E0B42E0A
:101D40008091160290911702A0911802B091190289
:101D50008093120290931302A0931402B093150281
:101D600080913A0390913B031A8A1B8A1C8A1D8A30
:101D70009A8389831C821B821C879A8689861D8789
:101D80000B87BE016A5E7F4FCE0101960E94A807B5
:101D900080933C036E897F8983E0769567958A9569
:101DA000E1F7660F771F660F771F072E000C880B71
:101DB000990B0E945C122FE632E143E85AE30E943D
:101DC0001113609322027093230280932402909354
:101DD000250280913A0390913B031FA218A619A6F1
:101DE0001AA69F8B8E8B198E188E19A33F8E2E8E5E
:101DF0001AA308A340913E0350913F036091400312
:101E000070914103CE0146960E942E0680913A03BE
:101E100090913B031A8A1B8A1C8A1D8A9A838983A4
:101E20001C821B821C8784E090E09A8789871D872B
:101E30000B87BE01655D7F4FCE0101960E94A8070A
:101E400080933C036BA57CA5072E000C880B990B97
:101E50000E945C122B013C0160914203709143038C
:101E600080914403909145030E945A129B01AC015A
:101E7000C301B2010E94B91120E030E04AE754E406
:101E80000E94B9119B01AC0120931E0230931F02E6
:101E9000409320025093210260912202709123020C
:101EA00080912402909125020E94111360931A02DE
:101EB00070931B0280931C0290931D022FB7F8941D
:101EC0006091330270913402809135029091360214
:101ED0002FBF0E945A126B017C01C0921602D09251
:101EE0001702E0921802F092190240901A025090E4
:101EF0001B0260901C0270901D022AE037ED43E245
:101F00005CE3C301B2010E940C1318160CF048C028
:101F10002091120230911302409114025091150247
:101F2000C701B6010E9447116B017C0120E030E03F
:101F30004AE754E40E94B9119B01AC0160912A0266
:101F400070912B0280912C0290912D020E944811D9
:101F500060932A0270932B0280932C0290932D029F
:101F6000A7019601C301B2010E94111320E030E0E5
:101F70004AE754E40E94B9119B01AC01609126022A
:101F80007091270280912802909129020E944811A5
:101F9000609326027093270280932802909329026F
:101FA00040912202509123026091240270912502F7
:101FB00022E081E992E00E94E10968E471E081E9B0
:101FC00092E00E94CF0A40911E0250911F02609140
:101FD00020027091210222E081E992E00E94E10951
:101FE00068E471E081E992E00E94CF0A40911A0210
:101FF00050911B0260911C0270911D0222E081E948
:1020000092E00E94E10968E471E081E992E00E94B7
:10201000CF0A4091260250912702609128027091C8
:10202000290222E081E992E00E94E10968E471E07E
:1020300081E992E00E94CF0A40912A0250912B023E
:1020400060912C0270912D0222E081E992E00E94C1
:10205000E1096AE471E081E992E00E9486096AEF91
:1020600070E080E090E00E94670182E00E94E00062
:102070003C01909331028093300283E00E94E000A3
:1020800090932F0280932E024091040150910501FC
:1020900041305105B9F46728A9F42091000130912D
:1020A00001012F5F3F4F30930101209300012091E8
:1020B0000001309101012630310524F050930101D7
:1020C000409300012091020130910301213031053C
:1020D00091F4892B81F410922A0210922B02109213
:1020E0002C0210922D0210922602109227021092BA
:1020F00028021092290280E00E94E30580910001ED
:10210000909101018330910509F48EC08CF58130E6
:10211000910509F44EC0029709F46BC0809130021A
:1021200090913102909305018093040180912E02D9
:1021300090912F029093030180930201A114B104A6
:1021400009F4FECD0E940302882309F4F9CD0E9410
:102150000000F6CD82E680934E0360E080E00E94AE
:102160005C056FEF88E00E945C0560E281E0D0CD05
:102170008430910509F46AC0059781F66EE971E033
:102180008AE493E00E94CF0A81E00E94E3056DE5B6
:1021900071E08AE493E00E94CF0A81E00E94E305A7
:1021A00040912A0250912B0260912C0270912D02D5
:1021B0001AC06DE471E08AE493E00E94CF0A81E0E6
:1021C0000E94E3056DE571E08AE493E00E94CF0A86
:1021D00081E00E94E3054091220250912302609128
:1021E00024027091250222E08AE493E00E94E10932
:1021F00095CF6EE671E08AE493E00E94CF0A81E019
:102200000E94E3056DE571E08AE493E00E94CF0A45
:1022100081E00E94E30540911E0250911F026091EF
:10222000200270912102DFCF6EE771E08AE493E033
:102230000E94CF0A81E00E94E30540911A0250916A
:102240001B0260911C0270911D02CDCF6EE871E0FF
:102250008AE493E00E94CF0A81E00E94E3056DE5E5
:1022600071E08AE493E00E94CF0A81E00E94E305D6
:102270004091260250912702609128027091290214
:10228000B2CF80913A0390913B030C94471450587D
:10229000BB27AA270E945F110C94D2120E94C4127D
:1022A00038F00E94CB1220F039F49F3F19F426F445
:1022B0000C94C1120EF4E095E7FB0C94BB12E92FCD
:1022C0000E94E31258F3BA17620773078407950751
:1022D00020F079F4A6F50C9405130EF4E0950B2E7E
:1022E000BA2FA02D0B01B90190010C01CA01A00168
:1022F0001124FF27591B99F0593F50F4503E68F1C3
:102300001A16F040A22F232F342F4427585FF3CF03
:10231000469537952795A795F0405395C9F77EF4D4
:102320001F16BA0B620B730B840BBAF09150A1F01D
:10233000FF0FBB1F661F771F881FC2F70EC0BA0FA3
:10234000621F731F841F48F4879577956795B7952B
:10235000F7959E3F08F0B0CF9395880F08F0992726
:10236000EE0F9795879508950E94971208F481E0E3
:1023700008950E94CD110C94D2120E94CB1258F0F5
:102380000E94C41240F029F45F3F29F00C94BB1264
:1023900051110C9406130C94C1120E94E31268F3BD
:1023A0009923B1F3552391F3951B550BBB27AA270E
:1023B00062177307840738F09F5F5F4F220F331F48
:1023C000441FAA1FA9F335D00E2E3AF0E0E832D010
:1023D00091505040E695001CCAF72BD0FE2F29D013
:1023E000660F771F881FBB1F261737074807AB07E5
:1023F000B0E809F0BB0B802DBF01FF2793585F4F5A
:102400003AF09E3F510578F00C94BB120C940613E1
:102410005F3FE4F3983ED4F3869577956795B7953B
:10242000F7959F5FC9F7880F911D9695879597F946
:102430000895E1E0660F771F881FBB1F62177307BF
:102440008407BA0720F0621B730B840BBA0BEE1FD4
:1024500088F7E09508950E94EB1288F09F5798F056
:10246000B92F9927B751B0F0E1F0660F771F881F99
:10247000991F1AF0BA95C9F714C0B13091F00E94B3
:102480000513B1E008950C940513672F782F882762
:10249000B85F39F0B93FCCF3869577956795B395DA
:1024A000D9F73EF490958095709561957F4F8F4F49
:1024B0009F4F0895E89409C097FB3EF4909580954E
:1024C000709561957F4F8F4F9F4F9923A9F0F92FFA
:1024D00096E9BB279395F695879577956795B79578
:1024E000F111F8CFFAF4BB0F11F460FF1BC06F5F5E
:1024F0007F4F8F4F9F4F16C0882311F096E911C070
:10250000772321F09EE8872F762F05C0662371F090
:1025100096E8862F70E060E02AF09A95660F771FA4
:10252000881FDAF7880F9695879597F90895990F80
:102530000008550FAA0BE0E8FEEF16161706E8078D
:10254000F907C0F012161306E407F50798F0621BAE
:10255000730B840B950B39F40A2661F0232B242B83
:10256000252B21F408950A2609F4A140A6958FEFA2
:10257000811D811D089597F99F6780E870E060E0F4
:1025800008959FEF80EC089500240A94161617060C
:1025900018060906089500240A9412161306140654
:1025A00005060895092E0394000C11F4882352F0B7
:1025B000BB0F40F4BF2B11F460FF04C06F5F7F4F6F
:1025C0008F4F9F4F089557FD9058440F551F59F056
:1025D0005F3F71F04795880F97FB991F61F09F3F10
:1025E00079F087950895121613061406551FF2CF39
:1025F0004695F1DF08C0161617061806991FF1CF89
:1026000086957105610508940895E894BB276627AF
:102610007727CB0197F908950E94971208F48FEF5E
:1026200008950E9424130C94D2120E94C41238F010
:102630000E94CB1220F0952311F00C94BB120C9445
:10264000C11211240C9406130E94E31270F3959F9B
:10265000C1F3950F50E0551F629FF001729FBB2799
:10266000F00DB11D639FAA27F00DB11DAA1F649F35
:102670006627B00DA11D661F829F2227B00DA11DE8
:10268000621F739FB00DA11D621F839FA00D611D6E
:10269000221F749F3327A00D611D231F849F600D8F
:1026A000211D822F762F6A2F11249F5750409AF0B8
:1026B000F1F088234AF0EE0FFF1FBB1F661F771F44
:1026C000881F91505040A9F79E3F510580F00C940F
:1026D000BB120C9406135F3FE4F3983ED4F3869547
:1026E00077956795B795F795E7959F5FC1F7FE2BAF
:1026F000880F911D9695879597F908950E949712D6
:10270000880B990B0895A1E21A2EAA1BBB1BFD0191
:102710000DC0AA1FBB1FEE1FFF1FA217B307E407C0
:10272000F50720F0A21BB30BE40BF50B661F771F18
:10273000881F991F1A9469F76095709580959095F8
:102740009B01AC01BD01CF010895EE0FFF1F059065
:10275000F491E02D09940F931F93CF93DF93823070
:10276000910510F482E090E0E0915903F0915A0352
:1027700030E020E0B0E0A0E0309799F42115310579
:1027800009F44AC0281B390B24303105D8F58A8159
:102790009B816115710589F1FB0193838283FE01A1
:1027A00011C0408151810281138148175907E0F01F
:1027B0004817590799F4109761F012960C931297E5
:1027C00013961C933296CF01DF91CF911F910F91F9
:1027D00008950093590310935A03F4CF211531053E
:1027E00051F04217530738F0A901DB019A01BD01EE
:1027F000DF01F801C1CFEF01F9CF90935A03809325
:102800005903CDCFFE01E20FF31F81939193225024
:10281000310939832883D7CF20915703309158034A
:10282000232B41F420910801309109013093580382
:10283000209357032091060130910701211531059E
:1028400041F42DB73EB740910A0150910B01241B72
:10285000350BE0915703F0915803E217F307A0F40A
:102860002E1B3F0B2817390778F0AC014E5F5F4FE6
:102870002417350748F04E0F5F1F509358034093BD
:102880005703819391939FCFF0E0E0E09CCFCF93EB
:10289000DF930097E9F0FC01329713821282A09136
:1028A0005903B0915A03ED0130E020E01097A1F4F4
:1028B00020813181820F931F20915703309158035B
:1028C0002817390709F061C0F0935803E0935703C4
:1028D000DF91CF910895EA01CE17DF07E8F54A812D
:1028E0005B819E0141155105B1F7E901FB83EA8344
:1028F00049915991C40FD51FEC17FD0761F48081F0
:1029000091810296840F951FE901998388838281C2
:1029100093819B838A83F0E0E0E012968D919C91F5
:1029200013970097B9F52D913C911197CD0102961F
:10293000820F931F209157033091580328173907AE
:1029400039F6309751F510925A0310925903B0930B
:102950005803A0935703BCCFD383C28340815181D6
:10296000840F951FC817D90761F44E5F5F4F8881A8
:102970009981480F591F518340838A819B8193839A
:1029800082832115310509F0B0CFF0935A03E0930B
:1029900059039ECFFD01DC01C0CF13821282D7CF35
:1029A00010E0C2E6D0E004C0FE010E94A51321960B
:1029B000C336D107C9F7F894FFCF01000100010029
:1029C00000005B0380000000000039029901C6018D
:1029D0008602F701D501E9010000000076074907EA
:1029E000A5071F0742072F07200700000000FC056E
:1029F0009901A507EE036E616E00696E66006F7641
:102A000066003B000D0A0054656E73696F6E2856B0
:102A100029203A20202000202020202020202020B3
:102A20002020202020202000496E74656E73697478
:102A300065284129203A20005075697373616E63DF
:102A400065285729203A2000456E65726769652818
:102A50004A29203A2020200054656D70732873297C
:082A6000203A20202020200074
:107E0000112484B714BE81FFF0D085E080938100F7
:107E100082E08093C00088E18093C10086E0809377
:107E2000C20080E18093C4008EE0C9D0259A86E02C
:107E300020E33CEF91E0309385002093840096BBD3
:107E4000B09BFECF1D9AA8958150A9F7CC24DD24C4
:107E500088248394B5E0AB2EA1E19A2EF3E0BF2EE7
:107E6000A2D0813461F49FD0082FAFD0023811F036
:107E7000013811F484E001C083E08DD089C08234E0
:107E800011F484E103C0853419F485E0A6D080C0E4
:107E9000853579F488D0E82EFF2485D0082F10E0AE
:107EA000102F00270E291F29000F111F8ED06801E7
:107EB0006FC0863521F484E090D080E0DECF843638
:107EC00009F040C070D06FD0082F6DD080E0C81688
:107ED00080E7D80618F4F601B7BEE895C0E0D1E017
:107EE00062D089930C17E1F7F0E0CF16F0E7DF06D8
:107EF00018F0F601B7BEE89568D007B600FCFDCFD4
:107F0000A601A0E0B1E02C9130E011968C91119780
:107F100090E0982F8827822B932B1296FA010C0160
:107F200087BEE89511244E5F5F4FF1E0A038BF0790
:107F300051F7F601A7BEE89507B600FCFDCF97BE46
:107F4000E89526C08437B1F42ED02DD0F82E2BD052
:107F50003CD0F601EF2C8F010F5F1F4F84911BD097
:107F6000EA94F801C1F70894C11CD11CFA94CF0C13
:107F7000D11C0EC0853739F428D08EE10CD085E9AC
:107F80000AD08FE07ACF813511F488E018D01DD067
:107F900080E101D065CF982F8091C00085FFFCCF94
:107FA0009093C60008958091C00087FFFCCF809118
:107FB000C00084FD01C0A8958091C6000895E0E648
:107FC000F0E098E1908380830895EDDF803219F02E
:107FD00088E0F5DFFFCF84E1DECF1F93182FE3DFCA
:107FE0001150E9F7F2DF1F91089580E0E8DFEE27F6
:047FF000FF270994CA
:027FFE00040479
:00000001FF
